:100000000C9428010C9443010C9443010C9443017B
:100010000C9443010C9443010C9443010C94430150
:100020000C9443010C9443010C9443010C9433133E
:100030000C9443010C9443010C9443010C94430130
:100040000C9443010C9443010C9443010C94430120
:100050000C9443010C9443010C9443010C94300F15
:100060000C9443010C9443010C9443010C94430100
:10007000ACDE48FD0FD00073686F77206D616300C0
:1000800073686F7720697000697020006D6163206C
:1000900000726573657400696F2073657420646411
:1000A0007200696F206765742064647200696F2054
:1000B00073657420706F727400696F2067657420B7
:1000C000706F727400696F206765742070696E00CC
:1000D000667332302073656E64006673323020724E
:1000E00065636569766500667332302077733330F7
:1000F000300088008F0C77009A0D8000310C8C0046
:10010000B80B9100F4089700CD0AA200740AAD0064
:10011000220AB900C909C5005F0BD0001F0BDA0025
:100120004509E700FA08000000006465673A2025E9
:10013000752E257520432C206879673A2025752572
:10014000252C2077696E643A2025752E2575206B45
:100150006D2F682C207261696E3A2025752C206302
:100160006F756E7465723A202575002530327825DA
:1001700030327825303278253032780A00257820E0
:10018000257820257800706F72742025643A20301D
:10019000782530327800257800706F7274202564DD
:1001A0003A203078253032780025780025782025CF
:1001B0007820257800706F72742025643A2030789A
:1001C000253032780025780025782025782025787C
:1001D0000025783A25783A25783A25783A25783AEC
:1001E00025780069702025752E25752E25752E25FC
:1001F000752F25752E25752E25752E25752C2067B6
:100200006174657761792025752E25752E25752EEB
:100210002575006D616320253032783A25303278BB
:100220003A253032783A253032783A253032783AE9
:10023000253032780025752E25752E25752E2575CD
:10024000004F4B007061727365206572726F7200AF
:1002500011241FBECFEFD0E1DEBFCDBF11E0A0E083
:10026000B1E0EAE2F7E602C005900D92AA32B107CA
:10027000D9F71CE0AAE2B1E001C01D92AF3BB10783
:10028000E1F70C9445010C940000CFEFD0E1DEBF04
:10029000CDBF789488E190E02FE00FB6F894A89550
:1002A000809360000FBE20936000A8950E9477089D
:1002B0000E9441040E9490080E9407130E941D089A
:1002C000A8950E94A606A8950E949A08A8950E9443
:1002D0003908A8950E94D114F3CFFC0190E030E0DA
:1002E0000DC08191492F482728E09CE840FB4695A6
:1002F0000EF449272A95D1F7942F3F5F361789F7D7
:10030000892F99270895EF92FF920F931F93CF9310
:10031000DF93CDB7DEB763970FB6F894DEBF0FBE9D
:10032000CDBF8C01790183E1A0E0B0E09E012F5F99
:100330003F4FF901182E0E9414330115110541F0A9
:10034000F80186E00190D9010D929D018150D1F70D
:100350006115710549F0FB0180819181A281B38112
:100360008F839887A987BA874115510549F0FA010B
:1003700080819181A281B3818B879C87AD87BE8765
:10038000E114F10449F0F70180819181A281B381E8
:100390008F87988BA98BBA8BFE01319620E030E0D5
:1003A0008191282798E08CE820FB26950EF42827D9
:1003B0009A95D1F73F5F323199F72B8B83E1A0E01B
:1003C000B0E0FE013196182E0E94193380E090E0D3
:1003D00063960FB6F894DEBF0FBECDBFDF91CF910D
:1003E0001F910F91FF90EF9008950F931F93182F77
:1003F000062F282F3327C9018F7190704B9784F4F3
:100400002076307085E0359527958A95E1F78091C3
:100410002A0199272817390719F0822F0E941D02F7
:100420002C981F71812F80680E948A08802F0E945B
:100430008A082C9A1F910F9108951F93182F63E03B
:100440008FE10E942C02612F63708FE10E94F50101
:1004500010932A011F9108950F931F93182F062FB1
:10046000282F3327C9018F7190704B9784F4207621
:10047000307095E0359527959A95E1F780912A019E
:1004800099272817390719F0822F0E941D022C98EE
:100490001F71812F806A0E948A08802F0E948A081B
:1004A0002C9A1F910F91089560E48FE10E94F5014D
:1004B00080E49CE90197F1F760E48FE10E942C024F
:1004C00064E08FE10E94F50108951F93182F2C9886
:1004D0008AE70E948A08812F0E948A082C9A1F911D
:1004E00008950F931F93182F062F282F3327C90124
:1004F0008F7190704B9784F42076307045E035957D
:1005000027954A95E1F780912A01992728173907FD
:1005100019F0822F0E941D022C981F71812F806478
:100520000E948A08802F0E948A082C9A1F910F919E
:1005300008950F931F938C01682F82E00E9471022F
:10054000012F1127602F83E00E9471021F910F91EC
:1005500008950F931F938C01682F80E00E94710211
:10056000012F1127602F81E00E9471021F910F91CE
:1005700008952C988AE30E948A0880E00E948A08E5
:100580002C9A992708951F93182F282F3327C901D4
:100590008F7190704B9784F42076307075E03595AC
:1005A00027957A95E1F780912A019927281739072D
:1005B00019F0822F0E941D022C98812F8F710E94AA
:1005C0008A0880E00E948A0817FF03C080E00E942A
:1005D0008A082C9A99271F9108952C988FEF0E94D2
:1005E0008A088DE10E94C30280FFFBCF2C9A0895F8
:1005F0000F931F938B01682F84ED0E947102602F6F
:1006000086ED0E947102012F1127602F87ED0E9455
:1006100071028AEE0E94C30280FDFBCF1F910F91F1
:1006200008950F931F93682F84ED0E94710261E07B
:1006300082ED0E94F5018AEE0E94C30280FDFBCF8D
:1006400061E082ED0E942C0288ED0E94C302082F17
:1006500089ED0E94C30211279927982F8827802BA4
:10066000912B1F910F9108950E94ED0260E088E0A8
:100670000E94710260E089E00E9471026FEF8AE0DF
:100680000E9471026FE08BE00E94710260E084E0E2
:100690000E94710260E185E00E94710260E08CE0DE
:1006A0000E94710260E08DE00E94710260E08EE0C5
:1006B0000E94710260E08FE00E9471021092B0010E
:1006C0001092AF0160E881EC0E942C026DE080EC9A
:1006D0000E94F50162E382EC0E94F50160E070E0A7
:1006E00080E00E94F80280E00E94110390FF06C0A3
:1006F00061E082EC0E94F50162E105C061E082ECFC
:100700000E942C0265E184EC0E94710262E186EC99
:100710000E9471026CE087EC0E94710264E88AEC2E
:100720000E94710262E08BEC0E94710260912F01C5
:1007300084EE0E9471026091300185EE0E94710288
:100740006091310182EE0E9471026091320183EE6C
:100750000E9471026091330180EE0E9471026091EB
:10076000340181EE0E94710262E17CE084E10E942A
:10077000F8026BED8BE10E94710262E170E082E1B0
:100780000E94F80264E08FE10E94F50160E88EE1CA
:100790000E94F50108950F931F9382E00E94C30207
:1007A000082F83E00E94C30211279927982F8827DA
:1007B000802B912B1F910F9108950F931F9380E031
:1007C0000E94C302082F81E00E94C30211279927CB
:1007D000982F8827802B912B1F910F9108950F93AD
:1007E0001F93CF93DF9314E68FE10E94C30283FF30
:1007F00004C011501F3F19F0F7CF1123E9F160E059
:1008000084E00E94710260E185E00E9471026091C3
:10081000FA0186E00E9471026091FA017091FB0179
:100820006050704F672F772787E00E94710280E049
:1008300090E10E94990280E00E946502C0E0D0E051
:100840000DED19E006C0F80181918F010E9465024B
:1008500021968091FA019091FB01C817D90798F36E
:1008600060E88FE10E94F50160E88FE10E942C02B0
:1008700068E08FE10E94F501DF91CF911F910F9108
:100880000895CF92DF92EF92FF920F931F93CF9331
:10089000DF93CDB7DEB724970FB6F894DEBF0FBE57
:1008A000CDBF0E94B0180E94C02583E10DED19E074
:1008B000A0E0B0E0F801182E0E94143362E1C801F4
:1008C0000E946D0168019091EF09891709F466C0D3
:1008D00046E050E060E770E08FE291E00E94BC2BC0
:1008E000D801EFE2F1E086E001900D928150E1F74E
:1008F0002AE030E03A83298380E095E09C838B8373
:100900003093DA092093D9099093DC098093DB09AD
:1009100089819A81AB81BC81F60186839783A08708
:10092000B1872FEF3FEF3A8329838FEF90E09C83CD
:100930008B833093D6092093D5099093D80980935F
:10094000D70989819A81AB81BC8182879387A487EB
:10095000B5871A8219821C821B82EE24FF24109212
:100960009E0910929D091092A00910929F098981F9
:100970009A81AB81BC8186879787A08BB18B0DED67
:1009800019E062E1C8010E946D01F601828B83E1EA
:10099000D701F801182E0E94193350C0AFE2B1E020
:1009A000F80186E001900D928150E1F78091E30912
:1009B0009091E409A091E509B091E60989839A83B1
:1009C000AB83BC8389819A819093DA098093D9099A
:1009D0008B819C819093DC098093DB098091E709EE
:1009E0009091E809A091E909B091EA0989839A8375
:1009F000AB83BC8389819A819093D6098093D50972
:100A00008B819C819093D8098093D7098091EB09C1
:100A10009091EC09A091ED09B091EE0989839A8338
:100A2000AB83BC8389819A8190939E0980939D09B1
:100A30008B819C819093A00980939F098EE00DED9E
:100A400019E0A3E1B0E0F801182E0E9414336DE024
:100A5000C8010E946D019091EA09891771F0109206
:100A6000AB011092AC011092AD011092AE018091D9
:100A7000A1018E7F8093A10119C08091DD09909121
:100A8000DE09A091DF09B091E0098093AB0190935A
:100A9000AC01A093AD01B093AE01A1EAB1E0F801C1
:100AA000349689E001900D928150E1F70E942D0F5C
:100AB0000E94340324960FB6F894DEBF0FBECDBF5C
:100AC000DF91CF911F910F91FF90EF90DF90CF902A
:100AD0000895EF92FF920F931F93CF93DF93CDB7BB
:100AE000DEB724970FB6F894DEBF0FBECDBF89E303
:100AF0000E94C302882309F41CC18091AF01909128
:100B0000B0010E94A9020E94B902082F0E94B902F6
:100B100011279927982F8827082B192B1093B0019C
:100B20000093AF018E010F5F1F4F78010E94B90241
:100B3000F80181938F01C7010496E817F907B1F70F
:100B400089819A819C01245030404297835792407A
:100B500008F0EFC03A8329836DEDE62E69E0F62EAA
:100B600000E010E007C00E94B902F70181937F0105
:100B70000F5F1F4F89819A8108171907A0F390937F
:100B8000FB018093FA018091E9099091EA090E94A2
:100B90001719F8E080309F0709F44FC0865098403D
:100BA00009F0A4C00E94D6258091FA019091FB0122
:100BB000892B09F49BC014E68FE10E94C30283FFD6
:100BC00004C011501F3F21F0F7CF112309F48EC04C
:100BD00060E084E00E94710260E185E00E947102A1
:100BE0006091FA0186E00E9471026091FA017091B1
:100BF000FB016050704F672F772787E00E947102DA
:100C000080E090E10E94990280E00E94650200E08D
:100C100010E04DEDE42E49E0F42E07C0F70181917C
:100C20007F010E9465020F5F1F4F8091FA01909132
:100C3000FB010817190790F34DC081E00E94911A3B
:100C40008091FA019091FB01892B09F44FC00E9419
:100C5000852414E68FE10E94C30283FF04C0115073
:100C60001F3F21F0F7CF112309F440C060E084E07A
:100C70000E94710260E185E00E9471026091FA01B8
:100C800086E00E9471026091FA017091FB01605050
:100C9000704F672F772787E00E94710280E090E114
:100CA0000E94990280E00E94650200E010E02DEDB4
:100CB000E22E29E0F22E07C0F70181917F010E9408
:100CC00065020F5F1F4F8091FA019091FB01081799
:100CD000190790F360E88FE10E94F50160E88FE169
:100CE0000E942C0268E08FE10E94F5016091AF0143
:100CF0007091B001CB0101978050904130F06FEFBF
:100D00008CE00E9471026FE00DC061508CE00E9487
:100D100071026091AF017091B00161507040672F16
:100D2000770F770B8DE00E94710260E48EE10E94E4
:100D3000F50124960FB6F894DEBF0FBECDBFDF914C
:100D4000CF911F910F91FF90EF900895CF92DF9276
:100D5000EF92FF920F931F93CF93DF93CDB7DEB740
:100D600024970FB6F894DEBF0FBECDBF89E30E9473
:100D7000C3021B9953C1882309F450C18CE10E941E
:100D8000C302182F60E88BE10E942C02C12EDD24E3
:100D9000C4FE06C083E10E94110381E10E94110399
:100DA000C3FE08C068E08CE10E942C026AE08DE17D
:100DB0000E942C02C6FE20C189E30E94C302882340
:100DC00009F41AC18091AF019091B0010E94A9026B
:100DD0000E94B902082F0E94B90211279927982F63
:100DE0008827082B192B1093B0010093AF018E01B7
:100DF0000F5F1F4F78010E94B902F80181938F01A4
:100E0000C7010496E817F907B1F789819A81049719
:100E10009A8389830E978357924008F0EDC000E0D3
:100E200010E08DEDE82E89E0F82E07C00E94B9028F
:100E3000F70181937F010F5F1F4F89819A81081706
:100E40001907A0F39093FB018093FA018091E909BF
:100E50009091EA090E941719F8E080309F0709F481
:100E60004FC08650984009F0A4C00E94D6258091BA
:100E7000FA019091FB01892B09F49BC014E68FE1E4
:100E80000E94C30283FF04C011501F3F21F0F7CF1F
:100E9000112309F48EC060E084E00E94710260E1D9
:100EA00085E00E9471026091FA0186E00E94710261
:100EB0006091FA017091FB016050704F672F7727A6
:100EC00087E00E94710280E090E10E94990280E038
:100ED0000E94650200E010E0BDEDEB2EB9E0FB2EB4
:100EE00007C0F70181917F010E9465020F5F1F4FCC
:100EF0008091FA019091FB010817190790F34DC0FA
:100F000081E00E94911A8091FA019091FB01892B56
:100F100009F44FC00E94852414E68FE10E94C302A9
:100F200083FF04C011501F3F21F0F7CF112309F4B4
:100F300040C060E084E00E94710260E185E00E94B0
:100F400071026091FA0186E00E9471026091FA01DB
:100F50007091FB016050704F672F772787E00E94E8
:100F6000710280E090E10E94990280E00E94650297
:100F700000E010E0FDEDEF2EF9E0FF2E07C0F701D5
:100F800081917F010E9465020F5F1F4F8091FA01DE
:100F90009091FB010817190790F360E88FE10E9418
:100FA000F50160E88FE10E942C0268E08FE10E9469
:100FB000F5016091AF017091B001CB0101978050B4
:100FC000904130F06FEF8CE00E9471026FE00DC035
:100FD00061508CE00E9471026091AF017091B0018C
:100FE00061507040672F770F770B8DE00E94710280
:100FF00060E48EE10E94F501C0FE06C061E08CE174
:101000000E942C020E943403C1FE04C062E08CE105
:101010000E942C0260E88BE10E94F50124960FB635
:10102000F894DEBF0FBECDBFDF91CF911F910F911E
:10103000FF90EF90DF90CF900895CF93DF93CAE0B9
:10104000D1E0A2EAB1E026E131E0E991F9918081B5
:101050008C93F901819191919F01FC018081FD01A7
:1010600084831196F1E0C231DF0779F7DF91CF91E8
:1010700008950F931F93CF93DF93CAE0D1E062E10D
:1010800071E0A2EAB1E046E151E009911991F8015D
:101090009081FB013191BF01232F209593238C91E7
:1010A0008223982BF8019083FA0101911191AF01ED
:1010B000F80180818323FD0194812923822BF8018B
:1010C00080831196F1E0C231DF07F9F6DF91CF910D
:1010D0001F910F910895E82FFF27EE0FFF1FEE5F7E
:1010E000FE4F0190F081E02D80819927089582EBD9
:1010F00084B984B1836084B980E185B985B18360A6
:1011000085B980E58CBD81E08DBD08950DB407FEE5
:10111000FDCF08958EBD0E9486088EB5992708954B
:101120008DE08093810086E891E090938900809320
:1011300088000895CF93DF93B19B53C080912B011A
:1011400090912C01019690932C0180932B010E9489
:10115000C01080912B0190912C016AE070E00E94F8
:10116000C932892B79F5C9E0D2E0D0930802C09347
:10117000070282E00E94911A8091FA019091FB018E
:10118000892B21F00E9485240E94EF03C054DF4F79
:1011900029E0C938D20749F7C1E6DCE0D093040260
:1011A000C093030285E00E94911A8091FA01909108
:1011B000FB01892B11F00E94EF0329968CE0CB3BB9
:1011C000D80761F780912B0190912C01845F9140A9
:1011D00031F40E94942510922C0110922B0182E090
:1011E00086BBDF91CF910895E0E0F0E0099580E0C3
:1011F00090E00895CF92DF92EF92FF920F931F93AA
:10120000C090F501D090F6018091F40182958F7025
:1012100081702091F9012F70A091F8010091F701E0
:10122000E091F401EF70E090F301DF92CF92992703
:101230009F938F9333273F932F93BB27BF93AF93F6
:1012400011271F930F93FF27FF93EF93FF24E7FCD2
:10125000F094FF92EF928AE291E09F938F935F93D5
:101260004F937F936F930E943A2C2DB73EB72C5E1D
:101270003F4F0FB6F8943EBF0FBE2DBF1F910F9189
:10128000FF90EF90DF90CF900895AF92BF92DF92E2
:10129000EF92FF920F931F93CF93DF937A015B013D
:1012A00020E000E010E057C0FF2793E0EE0FFF1FA3
:1012B0009A95E1F7DF01A354BE4F8C9186958695F0
:1012C000ED0169816295660F660F607C682BDF0116
:1012D000A254BE4F8C91869586958695ED014981E5
:1012E0004295440F407E482BDF01A154BE4F8C91A4
:1012F00082958F70ED0129812295207F282BE05463
:10130000FE4FA081A295A695A7708181880F880FB6
:10131000880F8A2B77277F936F9355275F934F937F
:1013200033273F932F9399279F938F938BE691E0D9
:101330009F938F93BF92AF920E94762C89E090E0AA
:10134000A80EB91E2D2DCDB7DEB72C960FB6F8948A
:10135000DEBF0FBECDBFE02F8091E401081758F427
:1013600089E0D82ED20E0F5F1F4F8D2D99278E1535
:101370009F0508F499CF1092E401822F9927DF91FD
:10138000CF911F910F91FF90EF90DF90BF90AF90A2
:101390000895EF92FF920F931F93CF93DF93CDB7F2
:1013A000DEB722970FB6F894DEBF0FBECDBF7B012C
:1013B0008A019E012F5F3F4F3F932F9329EA31E02F
:1013C0003F932F939F938F930E94A82C2DB73EB7E6
:1013D0002A5F3F4F0FB6F8943EBF0FBE2DBF019757
:1013E00011F529813A8124303105E8F4F901EF55EE
:1013F000FE4F858199279F938F933F932F9389E980
:1014000091E09F938F931F930F93FF92EF920E940F
:101410003A2C2DB73EB7265F3F4F0FB6F8943EBF2C
:101420000FBE2DBF02C08FEF9FEF22960FB6F8942C
:10143000DEBF0FBECDBFDF91CF911F910F91FF9007
:10144000EF900895CF93DF93CDB7DEB726970FB611
:10145000F894DEBF0FBECDBF9E012B5F3F4F3F9381
:101460002F939E012D5F3F4F3F932F939E012F5F40
:101470003F4F3F932F932CEA31E03F932F939F935D
:101480008F930E94A82C2DB73EB7265F3F4F0FB613
:10149000F8943EBF0FBE2DBF8230910529F48FEF27
:1014A00090E09E838D8302C0039799F4E981FA81CD
:1014B000E430F10570F42D81EF55FE4F822F8095B9
:1014C000958189239B812923822B858380E090E06D
:1014D00002C08FEF9FEF26960FB6F894DEBF0FBEC7
:1014E000CDBFDF91CF910895EF92FF920F931F939D
:1014F000CF93DF93CDB7DEB722970FB6F894DEBF58
:101500000FBECDBF7B018A019E012F5F3F4F3F93EE
:101510002F9325EC31E03F932F939F938F930E945D
:10152000A82C2DB73EB72A5F3F4F0FB6F8943EBFA9
:101530000FBE2DBF019711F529813A812430310565
:10154000E8F4F901EF55FE4F818199279F938F931E
:101550003F932F9385EB91E09F938F931F930F936E
:10156000FF92EF920E943A2C2DB73EB7265F3F4F75
:101570000FB6F8943EBF0FBE2DBF02C08FEF9FEF96
:1015800022960FB6F894DEBF0FBECDBFDF91CF918C
:101590001F910F91FF90EF900895CF93DF93CDB7F8
:1015A000DEB726970FB6F894DEBF0FBECDBF9E0103
:1015B0002B5F3F4F3F932F939E012D5F3F4F3F93F4
:1015C0002F939E012F5F3F4F3F932F9328EC31E0E5
:1015D0003F932F939F938F930E94A82C2DB73EB7D4
:1015E000265F3F4F0FB6F8943EBF0FBE2DBF82302F
:1015F000910529F48FEF90E09E838D8302C00397BD
:1016000099F4E981FA81E430F10570F42D81EF5508
:10161000FE4F822F8095918189239B812923822BE4
:10162000818380E090E002C08FEF9FEF26960FB697
:10163000F894DEBF0FBECDBFDF91CF910895CF9359
:10164000DF93CDB7DEB726970FB6F894DEBF0FBE97
:10165000CDBF9E012B5F3F4F3F932F939E012D5F88
:101660003F4F3F932F939E012F5F3F4F3F932F9309
:101670002DE731E03F932F939F938F930E94A82CE7
:101680002DB73EB7265F3F4F0FB6F8943EBF0FBE53
:101690002DBF039719F08FEF9FEF08C04D816B812D
:1016A00089819A810E947F1380E090E026960FB690
:1016B000F894DEBF0FBECDBFDF91CF910895EF92BA
:1016C000FF920F931F93CF93DF93CDB7DEB722978F
:1016D0000FB6F894DEBF0FBECDBF7B018A019E011D
:1016E0002F5F3F4F3F932F9326E931E03F932F9396
:1016F0009F938F930E94A82C2DB73EB72A5F3F4F30
:101700000FB6F8943EBF0FBE2DBF019711F589812A
:101710009A8184309105E8F40E946B0899279F9381
:101720008F9389819A819F938F9386E891E09F930D
:101730008F931F930F93FF92EF920E943A2C2DB735
:101740003EB7265F3F4F0FB6F8943EBF0FBE2DBF8A
:1017500002C08FEF9FEF22960FB6F894DEBF0FBE48
:10176000CDBFDF91CF911F910F91FF90EF90089522
:10177000CF92DF92EF92FF920F931F93CF93DF935D
:10178000CDB7DEB726970FB6F894DEBF0FBECDBF3C
:101790007C018CE090E00E94C32A8C01009709F440
:1017A00047C06C01065F1F4F1F930F9302501040FC
:1017B0001F930F93025010401F930F93025010403D
:1017C0001F930F93025010401F930F93025010402D
:1017D0001F930F9381ED91E09F938F93FF92EF9270
:1017E0000E94A82C2DB73EB7205F3F4F0FB6F8944C
:1017F0003EBF0FBE2DBF069701F5FE0131969E013B
:10180000295F3F4FD8018C9181930E5F1F4FE217E4
:10181000F307C1F7C6010E94662B20E030E040E0EC
:1018200050E060E070E0CE0101960E94830101C0AB
:101830008EEF992787FD909505C0C8010E94662B01
:101840008FEFF7CF26960FB6F894DEBF0FBECDBF51
:10185000DF91CF911F910F91FF90EF90DF90CF908C
:101860000895CF93DF93CDB7DEB72C970FB6F894DA
:10187000DEBF0FBECDBF8CE0A6E0B0E0FE0131962A
:10188000182E0E9414338C8599279F938F938B85F4
:1018900099279F938F938A8599279F938F93898503
:1018A00099279F938F93888599279F938F938F81F3
:1018B00099279F938F938E8199279F938F938D81E3
:1018C00099279F938F938C8199279F938F938B81D7
:1018D00099279F938F938A8199279F938F938981CB
:1018E00099279F938F9383EE91E09F938F935F93BC
:1018F0004F937F936F930E943A2C2DB73EB7225E91
:101900003F4F0FB6F8943EBF0FBE2DBF2C960FB6BB
:10191000F894DEBF0FBECDBFDF91CF910895AF9297
:10192000BF92CF92DF92EF92FF920F931F93CF93CC
:10193000DF93CDB7DEB72C970FB6F894DEBF0FBE9E
:10194000CDBF7C016E010894C11CD11CE114F104CF
:1019500021F468C00894E11CF11CD7018C918032FD
:10196000C9F388E090E00E94C32A8C01009709F433
:1019700059C05C010A5F1F4F1F930F930250104024
:101980001F930F93025010401F930F93025010406B
:101990001F930F9385E392E09F938F93FF92EF92B3
:1019A0000E94A82CEDB7FEB73C960FB6F894FEBF88
:1019B0000FBEEDBF049799F5C114D10461F0F60193
:1019C00096012C5F3F4FD8018C9181930E5F1F4F82
:1019D000E217F307C1F7C5010E94662B60E270E0D1
:1019E000C7010E942E2C7C01E4E0F0E0CE0EDF1E49
:1019F000CE010D96C816D90609F0A8CF9E01275F23
:101A00003F4FAE014B5F5F4FBE016F5F7F4F80E086
:101A100090E00E948301992787FD909505C0C80139
:101A20000E94662B8FEF9FEF2C960FB6F894DEBFC7
:101A30000FBECDBFDF91CF911F910F91FF90EF901F
:101A4000DF90CF90BF90AF9008956F927F928F926A
:101A50009F92AF92BF92CF92DF92EF92FF920F933D
:101A60001F93CF93DF937C015B013A01FC0101904E
:101A70000020E9F73197E81BF90B339718F480E061
:101A800090E049C0CC24DD240C2D1127000F111F3C
:101A9000000F111FF801EE50FF4FC591D491209710
:101AA00011F1CE010E94C92B4C010894C11CD11C1C
:101AB000AC01BE01C7010E94D22B892B29F7F80186
:101AC000EC50FF4F259134912115310561F0A301B0
:101AD000B501C701880D991DF90109952FEF8F3FB9
:101AE000920779F402C08FEF9FEFA114B10499F02F
:101AF000A30164E472E0C5010E94E92B8CE090E050
:101B00000AC0009741F4A30161E472E0C5010E949C
:101B1000E92B82E090E0DF91CF911F910F91FF9030
:101B2000EF90DF90CF90BF90AF909F908F907F907D
:101B30006F900895CF93DF93CDB7DEB726970FB69A
:101B4000F894DEBF0FBECDBF9E012F5F3F4F86E0F2
:101B5000A0E0B0E0F901182E0E9414338E8199277D
:101B60009F938F938D8199279F938F938C81992732
:101B70009F938F938B8199279F938F93F9018181F5
:101B800099279F938F93898199279F938F9383E1BF
:101B900092E09F938F935F934F937F936F930E94F5
:101BA0003A2C2DB73EB72E5E3F4F0FB6F8943EBF8E
:101BB0000FBE2DBF26960FB6F894DEBF0FBECDBF69
:101BC000DF91CF9108950F931F93CF93DF93E0910F
:101BD0000702F0910802EF016C96E459FF4F8081F3
:101BE00020E530E0281B310921153105C1F0409175
:101BF000FA015091FB012417350710F08A0101C04A
:101C000089016091050270910602A801CE010E942F
:101C1000052CFE01E05BFF4F8081800F8083C05B5D
:101C2000DF4F4881C055D04055276AE070E0CE01B3
:101C30000E94F82BFC01892B79F44091FA01509114
:101C4000FB016AE070E080910502909106020E941B
:101C5000F82B892B19F429C0108205C0C15BDF4F16
:101C60001882CF54D040BE016F5A7F4F4FE450E0EE
:101C7000CE010E94250D9C011816190674F4FC0172
:101C8000EC0FFD1FEF5AFF4F8AE08083CF55DF4FE7
:101C90002F5F3F4F2883C15AD04080E5FE0111924B
:101CA0008A95E9F7C05BDF4F1882DF91CF911F91D2
:101CB0000F9108958AE09DE80E94F9180895EF9227
:101CC000FF920F931F93CF93DF93E0910702F09160
:101CD00008028CE1E82EF12CEE0EFF1E809102022C
:101CE00086FF0FC0E459FF4F1082EF5AFF4F119249
:101CF00080E5D7011D928A95E9F711821082EE5B8B
:101D0000F0408091020280FF03C0E354FF4F108235
:101D10008091020281FF6EC0E0910702F0910802FB
:101D2000EF016C96E459FF4F808120E530E0281BDD
:101D3000310921153105C1F04091FA015091FB01A3
:101D40002417350710F08A0101C08901609105024E
:101D500070910602A801CE010E94052CFE01E05BF5
:101D6000FF4F8081800F8083C05BDF4F4881C0556B
:101D7000D04055276AE070E0CE010E94F82BFC01AC
:101D8000892B79F44091FA015091FB016AE070E0EF
:101D900080910502909106020E94F82B892B19F47C
:101DA00029C0108205C0C15BDF4F1882CF54D040DC
:101DB000BE016F5A7F4F4FE450E0CE010E94250DC7
:101DC0009C011816190674F4FC01EC0FFD1FEF5A64
:101DD000FF4F8AE08083CF55DF4F2F5F3F4F28832F
:101DE000C15AD04080E5FE0111928A95E9F7C05BA7
:101DF000DF4F188280910202992782FD08C081FD81
:101E000006C080FD04C086FD02C083FF12C081EAC7
:101E100090E0E80EF91ED7016C91EFE5FFEFEE0EB2
:101E2000FF1E662331F07727C7018F5A9F4F0E940C
:101E30001B19DF91CF911F910F91FF90EF900895A3
:101E40000895E0910702F0910802848195818A50FB
:101E50009D4811F40E945F0E08950E945A0E089545
:101E60001F920F920FB60F9211247F928F929F9222
:101E7000AF92BF92CF92DF92EF92FF920F931F9398
:101E80002F933F934F935F936F937F938F939F9382
:101E9000AF93BF93EF93FF937090B2001092B20094
:101EA0008091E501882309F0E6C08091BA018A3368
:101EB00008F0E1C0872D8152893208F046C0909128
:101EC0002E01892F8152893208F03FC0472D5527B6
:101ED000292F3327CA01821B930B85349105ACF55A
:101EE000241B350B2534310584F510922E011092F8
:101EF000BB018090B2019090B301A090B401B0906A
:101F0000B501C090B601D090B701E090B801F09053
:101F1000B90101E0282D392D4A2D5B2D6C2D7D2D29
:101F20008E2D9F2D0E94382A2093B2013093B30149
:101F30004093B4015093B5016093B6017093B7011B
:101F40008093B8019093B9016EC0872D8A54803276
:101F500008F06FC090912E01892F8A54803208F0CA
:101F600068C0472D5527292F3327CA01821B930BA1
:101F7000853491050CF05DC0241B350B25343105EB
:101F80000CF057C010922E011092BB018090B2014C
:101F90009090B301A090B401B090B501C090B6018B
:101FA000D090B701E090B801F090B90101E0282D80
:101FB000392D4A2D5B2D6C2D7D2D8E2D9F2D0E9450
:101FC000382A2093B2013093B3014093B401509367
:101FD000B5016093B6017093B7018093B8019093F7
:101FE000B901A090B201B090B301C090B401D090FB
:101FF000B501E090B601F090B7010091B8011091E1
:10200000B9012A2D21602093B201B092B301C09290
:10201000B401D092B501E092B601F092B7010093FD
:10202000B8011093B9018091BA018F5F8093BA0112
:1020300022C08091BB018430B8F01092BB01109295
:10204000BA0110922E011092B2011092B3011092B7
:10205000B4011092B5011092B6011092B70110921E
:10206000B8011092B90107C070922E018091BB0196
:102070008F5F8093BB018091F1018F3408F064C0C1
:1020800090912D01892F8A558B3530F4872D8451FD
:102090008D3310F490E00AC094519D3330F4872DB5
:1020A0008A558B3510F491E001C09FEF8091F001CB
:1020B00080FD27C0992369F49091F0019E7F9E5F77
:1020C0008091F0018170892B8093F00110922D0195
:1020D0003BC09130B9F58091F0018695992708971A
:1020E00044F08091F00181608093F00110922D0105
:1020F00002C070922D018091F00181708093F001F7
:1021000023C097FD1FC0E091F1013091F1019130A2
:1021100089F4E695E695E695FF27EF54FE4F25A94D
:10212000377081E090E002C0880F991F3A95E2F77E
:10213000282B25AB10922D018091F1018F5F8093A8
:10214000F10102C070922D01FF91EF91BF91AF910B
:102150009F918F917F916F915F914F913F912F91BF
:102160001F910F91FF90EF90DF90CF90BF90AF90B5
:102170009F908F907F900F900FBE0F901F9018959B
:102180008091E501882329F08091E50181508093B9
:10219000E50108952F923F924F925F926F927F9246
:1021A0008F929F92AF92BF92CF92DF92EF92FF9267
:1021B0000F931F93CF93DF93CDB7DEB728970FB65A
:1021C000F894DEBF0FBECDBF8091E60184FF06C24A
:1021D0008091E70181FF02C28091E70186FFFEC185
:1021E0008091E80183FFFAC18091E90180FFF6C187
:1021F0008091E90185FFF2C18091EA0182FFEEC181
:102200008091EA0187FFEAC18091EB0184FFE6C17A
:102210008091EC0181FFE2C18091EC0186FFDEC17B
:102220008091ED0183FFDAC18091EE0180FFD6C17C
:102230008091EE0185FFD2C18091EF0182FFCEC176
:102240008091E6018F70873009F0C8C12091E601C6
:102250002F708091E6018295869587709090E701B6
:1022600031E09322990C990C990C982AF090E7018F
:10227000F694F6944FE0F4228091E701881F8827B6
:10228000881F9091E8019770990F982B5091E80161
:1022900052955F705A83E090E901E694E4228091C0
:1022A000E9018295869586958370C090EA0163E086
:1022B000C622CC0CCC0CC82A2090EA012694269485
:1022C000269424227091EB017F707B838091EB0137
:1022D000829586958770D090EC01D322DD0CDD0CC1
:1022E000DD0CD82A4090EC0146944694442280911B
:1022F000EC01881F8827881F4091ED014770440F2B
:10230000482B8091ED0182958F708C837090EE0147
:102310007694EFE07E228091EE01829586958695F7
:1023200083703091EF013370330F330F382B1091DE
:10233000E6011F708091E601829586958770709105
:10234000E7017170770F770F770F782B5090E701C7
:10235000569456945E228091E701881F8827881F33
:102360000091E8010770000F082B3090E8013694C7
:102370003694369436948090E90186948E2280912A
:10238000E9018295869586958370F091EA01F37054
:10239000FF0FFF0FF82BFF83A090EA01A694A694ED
:1023A000A694AE226090EB016E228091EB018295A3
:1023B000869587705091EC015170550F550F550F50
:1023C000582B58875091EC01569556955F70809127
:1023D000EC01881F8827881FA091ED01A770AA0F24
:1023E000A82BB090ED01B694B694B694B6946091D3
:1023F000EE0166956F708091EE01829586958695C7
:102400008370B091EF01B370BB0FBB0FB82B9F254A
:102410009E2592259D259427972529258A81282761
:102420002C25EB812E272425FC812F27232792178B
:1024300009F0D4C08091EF018695869586958F70BE
:10244000170F130D3F81130F160D150F1B0D1B0FCB
:10245000050D080D0A0D4885040F0A0F060F0B5FC6
:10246000100F1F70212F332799272817390709F0DC
:10247000B5C09091E701969596959F708091F40173
:10248000807F892B8093F4018091E701881F882742
:10249000881F9091E8019770990F982B8091E8011F
:1024A00082958F70AAE0B0E08A9F802D1124890F59
:1024B0008093F3019091E6019295969597708091A3
:1024C000E7018170880F880F880F892B90E081FDCC
:1024D00091E09295907F8091F4018F7E892B80937B
:1024E000F4012091E6012295269527708091E7015D
:1024F0008170880F880F880F822B992788709070C1
:10250000892B29F08091F30181958093F30120912B
:10251000E90126952F709091E901929596959695EF
:1025200093708091EA018370880F880F892B8A9FAE
:10253000802D1124820F8093F7019091EA019695E6
:10254000969596959F708091F901807F892B809355
:10255000F9012091EB012F709091EB0192959695E6
:1025600097708091EC018170880F880F880F892BFC
:102570008A9F802D1124820F8093F8015091EC01E5
:102580005695569559835F704091ED0142954F7075
:102590002091EC01221F2227221F8091ED018770DC
:1025A000880F822B99278A9F90018B9F300D9A9FCD
:1025B000300D1124642F772784E690E0FC016E9F94
:1025C000C0016F9F900D7E9F900D1124850F911D6E
:1025D000280F391F3093F6012093F50128960FB686
:1025E000F894DEBF0FBECDBFDF91CF911F910F9149
:1025F000FF90EF90DF90CF90BF90AF909F908F9023
:102600007F906F905F904F903F902F900895FF9232
:102610000F931F9301EB11E081E0F82EF092B101CE
:10262000229A2A9844E350E060E070E0C8010196E5
:102630000E94242C23982B9888E580BF1092B2002A
:102640001092B00085E08093B100F092700044E1F8
:1026500050E060E070E0C801C5960E94242C1F91F4
:102660000F91FF9008951F920F920FB60F921124B1
:102670002F933F934F935F936F937F938F939F938A
:10268000AF93BF93EF93FF938091BA018A3321F404
:102690008091E501882351F01092BA0148E050E0A2
:1026A00060E070E082EB91E00E94242C8091F101C7
:1026B0008F34A1F01092F1018091F0018E7F809310
:1026C000F0018091F00181708093F0014AE050E0C8
:1026D00060E070E086EE91E00E94242CFF91EF9183
:1026E000BF91AF919F918F917F916F915F914F912A
:1026F0003F912F910F900FBE0F901F9018950F9341
:102700001F93CF93DF93EC01162F642F00E042C19B
:102710002A9A80ED97E0FC013197F1F72A9801970A
:10272000F1F72F5F2C30A1F72A9A88EB9BE0FC0190
:102730003197F1F72A980197F1F78D2F9927782F84
:1027400027E041E050E0A8EBBBE0E0EDF7E0CA0194
:10275000022E02C0880F991F0A94E2F7872339F0EE
:102760002A9ACD010197F1F72A98CD0106C02A9A3D
:10277000CF010197F1F72A98CF010197F1F7215086
:1027800030F7872F082E82958025082E869586950E
:1027900080259927019681FF04C02A9A88EB9BE047
:1027A00003C02A9A80ED97E0FC013197F1F72A984F
:1027B0000197F1F73C2F27E041E050E0A8EBBBE0A8
:1027C000E0EDF7E0CA01022E02C0880F991F0A94BB
:1027D000E2F7832339F02A9ACD010197F1F72A987D
:1027E000CD0106C02A9ACF010197F1F72A98CF01AF
:1027F0000197F1F7215030F7832F082E829580251D
:10280000082E8695869580259927019681FF04C01C
:102810002A9A88EB9BE003C02A9A80ED97E0FC019E
:102820003197F1F72A980197F1F727E081E090E0DE
:10283000022E02C0880F991F0A94E2F7812321F02B
:102840002A9A88EB9BE003C02A9A80ED97E0FC016E
:102850003197F1F72A980197F1F7215038F7812F36
:10286000082E82958025082E8695869580259927A5
:10287000019681FF04C02A9A88EB9BE003C02A9A44
:1028800080ED97E0FC013197F1F72A980197F1F775
:1028900027E081E090E0022E02C0880F991F0A9481
:1028A000E2F7862321F02A9A88EB9BE003C02A9A5C
:1028B00080ED97E0FC013197F1F72A980197F1F745
:1028C000215038F7862F082E82958025082E869570
:1028D000869580259927019681FF04C02A9A88EB66
:1028E0009BE003C02A9A80ED97E0FC013197F1F755
:1028F0002A980197F1F73A5F360F272F210F230F00
:1029000037E041E050E0A8EBBBE0E0EDF7E0CA01C2
:10291000032E02C0880F991F0A94E2F7822339F030
:102920002A9ACD010197F1F72A98CD0106C02A9A7B
:10293000CF010197F1F72A98CF010197F1F73150B4
:1029400030F7022E22952025022E26952695202549
:10295000822F9927019681FF04C02A9A88EB9BE079
:1029600003C02A9A80ED97E0FC013197F1F72A988D
:102970000197F1F72A9A80ED97E0FC013197F1F782
:102980002A980197F1F784EF91E00197F1F70F5F33
:10299000033011F020E0BCCEDF91CF911F910F9159
:1029A00008952F923F924F925F926F927F928F92F3
:1029B0009F92AF92BF92CF92DF92EF92FF920F93CE
:1029C0001F93CF93DF93CDB7DEB725970FB6F8945B
:1029D000DEBF0FBECDBF8091BA018A3309F021C19D
:1029E0009091B7019295969597708091B801880F54
:1029F000880F880F282F292B9091B80192959695D2
:102A000097708091B9018370880F880F880F382FD5
:102A1000392B2130310509F0F2C08091B601829541
:102A2000869587702091B701220F220F220F282B45
:102A3000022E22952025022E26952695202590915E
:102A4000B60192959F708091B50182958F70F0913B
:102A5000B601F295F07FF82B0F2EF295F0250F2E90
:102A6000F695F695F025F090B501F694F694F69467
:102A700081E0F8228091B401869586958695E09153
:102A8000B501E295EE0FE07EE82B0E2EE295E025F3
:102A90000E2EE695E695E0250091B4010695069583
:102AA00001708091B301869586957091B4017295FD
:102AB000770F770F707C782B072E72957025072E75
:102AC0007695769570251091B301169511708091C9
:102AD000B20186955091B301579555275795582BBC
:102AE000052E52955025052E569556955025E09069
:102AF000B20181E0E8228091B601829586958770C7
:102B00006091B701660F660F660F682B8091B50163
:102B100082958F70B091B601B295B07FB82B80913D
:102B2000B401869586958695A091B501A295AA0FC8
:102B3000A07EA82B8091B301869586954091B40123
:102B40004295440F440F407C482B33272F5F3F4F63
:102B500035952795922790FD52C08F2F9927019682
:102B60009595879581709070F81609F048C08E2F62
:102B7000992701969595879581709070081709F0AF
:102B80003EC0872F99270196959587958170907003
:102B90001817A9F5852F9927019695958795817026
:102BA0009070E81661F58091B20186959091B3011D
:102BB000979599279795982B4A0F6B0F6A5F460F49
:102BC0004917E9F440E250E06CEB71E084EC91E0ED
:102BD0000E94122CECEBF1E0DF011A9788E00D90D7
:102BE00001928150E1F78091E401853028F48091D1
:102BF000E4018F5F8093E40186E08093E501109209
:102C0000B2011092B3011092B4011092B50110926A
:102C1000B6011092B7011092B8011092B90110924A
:102C2000BA018091F1018F3409F01CC28091E60154
:102C300084FF09C28091E70181FF05C28091E7010D
:102C400086FF01C28091E80183FFFDC18091E90107
:102C500080FFF9C18091E90185FFF5C18091EA010A
:102C600082FFF1C18091EA0187FFEDC18091EB0104
:102C700084FFE9C18091EC0181FFE5C18091EC0105
:102C800086FFE1C18091ED0183FFDDC18091EE01FE
:102C900080FFD9C18091EE0185FFD5C18091EF0100
:102CA00082FFD1C18091E6018F70873009F0CBC1DE
:102CB0002091E6012F708091E601829586958770BC
:102CC0007091E7017170770F770F770F782BE09194
:102CD000E701E695E695EF70EA838091E701881FAA
:102CE0008827881F9091E8019770990F982BE090A2
:102CF000E801E694E694E694E694F091E901F6950D
:102D0000FF70F9838091E90182958695869583709D
:102D10006091EA016370660F660F682B2090EA01EC
:102D20002694269426948FE02822F090EB01F82236
:102D30008091EB018295869587705091EC015170DE
:102D4000550F550F550F582BE091EC01E695E69580
:102D5000EF70ED838091EC01881F8827881F4091D8
:102D6000ED014770440F482BF091ED01F295FF7093
:102D7000FB838091EE0186958F708C838091EE01AC
:102D800082958695869583703091EF013370330F6D
:102D9000330F382B1091E6011F708091E601829568
:102DA00086958770B090E701E1E0BE22BB0CBB0CBA
:102DB000BB0CB82A4090E70146944694FFE04F22AE
:102DC0008091E701881F8827881F0091E80107701C
:102DD000000F082B3090E8013694369436943694E0
:102DE0006090E90166946F228091E9018295869551
:102DF00086958370C090EA01E3E0CE22CC0CCC0C27
:102E0000C82A7090EA017694769476947F22509046
:102E1000EB015F228091EB01829586958770D090BF
:102E2000EC01F1E0DF22DD0CDD0CDD0CD82A909006
:102E3000EC01969496948FE098228091EC01881F83
:102E40008827881FA091ED01A770AA0FA82B80905A
:102E5000ED018694869486948694A090EE01A694C3
:102E6000EFE0AE228091EE01829586958695837083
:102E7000B091EF01B370BB0FBB0FB82BFA819F2746
:102E800089819827922595279427EC819E272727CB
:102E90002E2526272F25FD812F278B8128272327C5
:102EA000921709F0D0C08091EF018695869586959E
:102EB0008F701B0D130D1C0D150D190D180D1B0F0B
:102EC000040D060D070D0D0D0A0F0A0D0B5F100FF7
:102ED0001F70212F332799272817390709F0B3C00E
:102EE0009091E701969596959F708091F401807F6F
:102EF000892B8093F4018091E701881F8827881F20
:102F00009091E8019770990F982B8091E801829534
:102F10008F70EAE0F0E08E9F802D1124890F80935E
:102F2000F3019091E6019295969597708091E70153
:102F30008170880F880F880F892B90E081FD91E0C8
:102F40009295907F8091F4018F7E892B8093F4017C
:102F50002091E6012295269527708091E7018170E6
:102F6000880F880F880F822B992788709070892B83
:102F700029F08091F30181958093F3012091E9017B
:102F800026952F709091E90192959695969593705C
:102F90008091EA018370880F880F892B8E9F802D86
:102FA0001124820F8093F7019091EA0196959695EE
:102FB00096959F708091F901807F892B8093F9010C
:102FC0002091EB012F709091EB019295969597705F
:102FD0008091EC018170880F880F880F892B8E9F5C
:102FE000802D1124820F8093F8016091EC01669589
:102FF00066956F704091ED0142954F702091EC0104
:10300000221F2227221F8091ED018770880F822BBB
:1030100099278E9F90018F9F300D9E9F300D112418
:10302000552784E690E0FC014E9FC0014F9F900D14
:103030005E9F900D1124860F911D280F391F30932C
:10304000F6012093F5014AE050E060E070E086EE82
:1030500091E00E94242C8091F0018E7F8093F001FA
:103060001092F10125960FB6F894DEBF0FBECDBFCA
:10307000DF91CF911F910F91FF90EF90DF90CF9054
:10308000BF90AF909F908F907F906F905F904F9088
:103090003F902F90089590933601809335010895C5
:1030A000FC018381860F80930102272F33278281C1
:1030B000820F8093000241814093FF01E081E09301
:1030C000FE0199278217930748F4842F8F5F80931E
:1030D000FF01882319F4EF5FE093FE018091010264
:1030E000992770708617970798F4809100028F5F78
:1030F00080930002882361F48091FF018F5F8093A9
:10310000FF01882329F48091FE018F5F8093FE01E7
:103110000895DC01460F571F41505040FB010EC07F
:1031200080819927982F88272181820F911DA80FD0
:10313000B91FA817B90708F411963296E417F507D6
:1031400078F3E417F50751F480819927982F8827A1
:10315000A80FB91FA817B90708F41196CD01089553
:1031600010923D01E9E8F9E01192119289E0ED3900
:10317000F807D1F710923D01E2E2F2E01082E0544C
:10318000FF4F89E0E23AF807C9F780E094E09093B6
:103190003C0180933B0110923D01E5E6FCE0118289
:1031A000108239968CE0EF3BF807C9F78AE08093EC
:1031B0003D010895BC0110923D0140E020E030E067
:1031C000E9E8F9E0DF01808191818617970729F40A
:1031D00040933D011D921C920895422F4F5F2F5F37
:1031E0003F4F129632962A30310569F740933D01E0
:1031F0000895BC0110923D0140E020E030E0E9E894
:10320000F9E0DF0180819181892B29F440933D0110
:103210006D937C930895422F4F5F2F5F3F4F12961F
:1032200032962A30310571F740933D010895292FD8
:10323000382FC90108959C01AB011616170674F4C6
:103240007093600C60935F0C8091FC019091FD0184
:103250002817390719F0B9010E94052C08950F931A
:103260001F93AB01BC0180E090E00E948918092FF8
:10327000182FC8011F910F9108950F931F93CF939B
:10328000DF93EC0120913B0130913C012F5F3F4FD8
:103290008DE72030380710F020E030E1432F522F27
:1032A000A0E0E5E6FCE0808191818417950771F349
:1032B000AF5F3996AA30B9F730933C0120933B01B8
:1032C00010923D01B0E040E050E0E5E6FCE0808196
:1032D0009181892B51F4B0933D0189E0489FF00121
:1032E0001124EF59F34F71F424C0B42FBF5F4F5F27
:1032F0005F4F39964A30510551F7B0933D01E0E0F8
:10330000F0E017C0032F122F1583048377836683A1
:10331000209729F4108211821282138208C08881BA
:103320009981918380838A819B819383828380E4C6
:103330008087CF01DF91CF911F910F910895EF9278
:10334000FF920F931F93CF93DF938C0120913B014A
:1033500030913C012F5F3F4F8DE72030380710F050
:1033600020E030E1432F522FE9E0F2E0A1E0818D2F
:10337000882329F0848195818417950759F38A2F32
:103380008F5FE054FF4F8B3011F0A82FF0CF3093B8
:103390003C0120933B0110923D01E0E0F0E090E021
:1033A00041E0A9E0B2E0ED01898D882321F49093FA
:1033B0003D01FD0117C0873041F4309729F0ED0140
:1033C0009A8D828D891708F4FD01842F8F5FA05498
:1033D000BF4F8B3019F0942F482FE5CF40933D011C
:1033E000309781F182E0818F8091370184878091CD
:1033F0003801858780913901868780913A018787D6
:103400008AE492E0938B828B958B848B81E090E0B1
:10341000918B808B138E81E0828F83E0808F168A60
:1034200080E1878BE32EF22EF582E4827783668338
:10343000D8018D919C9191838083E8018A819B8141
:1034400093838283CF01DF91CF911F910F91FF90E2
:10345000EF900895CF93DF9344E150E06BEE79E075
:1034600080E090E00E948918009719F4CFEFDFEF19
:1034700002C0C92FD82FCE01DF91CF9108950F93AD
:103480001F93CF93DF938091ED099927982F882779
:103490002091EE09820F911D8C010451104048E0EB
:1034A00050E067EF79E00E970E948918A8016FEF4E
:1034B00079E00E948918009719F4CFEFDFEF02C07E
:1034C000C92FD82FCE01DF91CF911F910F91089571
:1034D0000F931F93CF93DF938091ED099927982F36
:1034E00088272091EE09820F911D8C010451104014
:1034F00048E050E067EF79E003970E948918A8013F
:103500006FEF79E00E948918009719F4CFEFDFEF91
:1035100002C0C92FD82FCE01DF91CF911F910F91FB
:1035200008956F927F928F929F92AF92BF92CF92A7
:10353000DF92EF92FF920F931F93CF93DF93C0918F
:103540000702D0910802843009F4ACC223E13AE0CA
:1035500030930602209305023093FD012093FC0175
:10356000833069F4898D8F70833011F00C946A2454
:1035700088899989892B11F00C946A2499C082302A
:1035800009F09AC080913A018F5F80933A018823B5
:1035900099F4809139018F5F80933901882361F418
:1035A000809138018F5F80933801882329F48091BE
:1035B00037018F5F809337011092FB011092FA015F
:1035C0001092600C10925F0C298D273011F025307D
:1035D00051F48A8D8F5F8A8F883711F00C946A249A
:1035E000198E0C946A24222311F40C946A2488897D
:1035F0009989892B09F457C08A8D81508A8F8F3F12
:1036000011F00C946A243B8D383029F0215022307F
:1036100048F4353039F4198E80E8809302020E9414
:10362000210F6AC7353010F080E307C083E090E0D7
:1036300002C0880F991F3A95E2F78A8F8B8D8F5FB2
:103640008B8F8091C7099091C80901969093C80902
:103650008093C709898D99278F7090708330910569
:10366000E1F0843091054CF48130910509F4A4C453
:10367000029711F00C946A240DC08630910509F46C
:10368000AEC68830910509F4AAC6049711F00C94CF
:103690006A24A5C610920C0A92C484E080930202A8
:1036A0000E94210F5FC72F70233011F00C946A2401
:1036B00088E08093020213C7853021F5E091030270
:1036C000F091040284819581892B11F40C946A2471
:1036D0001092080210920702C9010C9790930602FB
:1036E000809305029093FD018093FC011092600C81
:1036F00010925F0C1092FB011092FA0188E0809307
:103700000202CEC18091A3099091A40901969093E1
:10371000A4098093A309B8EDEB2EBFEFFB2EE20EB8
:10372000F31E8091EB098534A1F08091A10990915D
:10373000A20901969093A2098093A1098091A709FB
:103740009091A80901969093A8098093A7090C94D9
:103750006A248091ED099927382F22278091EE095C
:10376000280F311D8091FA019091FB018217930778
:1037700010F40C946A243093FB012093FA01809199
:10378000F10999278F739070892B21F48091F209A8
:103790008823A1F08091A1099091A20901969093AC
:1037A000A2098093A1098091AD099091AE0901967B
:1037B0009093AE098093AD090C946A242091D909A5
:1037C0003091DA092115310531F48091DB099091AE
:1037D000DC09892BE9F08091FB099091FC098217A3
:1037E000930759F42091FD093091FE098091DB097E
:1037F0009091DC092817390759F08091A10990911F
:10380000A20901969093A2098093A1090C946A24BD
:1038100044E150E06BEE79E080E090E00E9489188E
:103820000097C9F0092F182F0F5F1F4FA1F080914B
:10383000A1099091A20901969093A2098093A109F0
:103840008091AF099091B00901969093B00980934F
:10385000AF090C946A248091F409863009F4A7C159
:10386000813109F472C08130A1F08091A109909159
:10387000A20901969093A2098093A1098091B109B0
:103880009091B20901969093B2098093B1090C947A
:103890006A248091B5099091B60901969093B60972
:1038A0008093B5098091FF098830A1F08091B30918
:1038B0009091B40901969093B4098093B3098091D3
:1038C000B9099091BA0901969093BA098093B90900
:1038D0000C946A241092FF098091010A9091020AC7
:1038E000EFEF873F9E0710F0099601C0089690936E
:1038F000020A8093010A8091F7099091F809909348
:10390000FC098093FB098091F9099091FA09909341
:10391000FE098093FD098091D9099091DA0990936D
:10392000F8098093F7098091DB099091DC09909365
:10393000FA098093F9098091B7099091B809019625
:103940009093B8098093B709BBC78091FA01909111
:10395000FB014C979093FB018093FA01C7E0DAE0FA
:10396000D0930602C09305028091050A9091060A41
:10397000892BB1F18091ED099927982F8827209103
:10398000EE09820F911D8C010451104048E050E077
:10399000BE016051704003970E948918A801BE01C2
:1039A000685070400E9489180097D1F0A92EB82E57
:1039B000FFEFAF16FFEFBF0699F08091CD09909110
:1039C000CE0901969093CE098093CD098091D309B9
:1039D0009091D40901969093D4098093D3097AC722
:1039E00081E69CE09093040280930302FC01C09165
:1039F000010AD091020AA091FF09B091000A6091DA
:103A0000F7097091F8094091F9095091FA098481F8
:103A10009581009729F1C817D90711F586819781FB
:103A2000009719F0A817B907D9F420813181211521
:103A3000310529F482819381892B51F41CC01FEF39
:103A40002F3F310729F4828193818F5F9F4F99F037
:103A50006217730729F4828193814817590759F037
:103A60003996F0930402E09303022CE0EB3BF2075B
:103A700008F030C7CCCF109208021092070282E003
:103A80008093020287E09AE09093060280930502F9
:103A90009093FD018093FC011092600C10925F0CDA
:103AA0000E94200F60915F0C7091600C6115710590
:103AB00009F410C7CB014C969093FB018093FA0157
:103AC000892F99278093ED094091FA014093EE09DF
:103AD000E0910302F091040220852093F30921E193
:103AE0002093F4099B01285F3F4F832E922E9092E2
:103AF000040A8092030A1092060A1092050A248191
:103B000035813093000A2093FF0926813781309355
:103B1000020A2093010A2091D9093091DA093093E1
:103B2000F8092093F7092091DB093091DC093093E3
:103B3000FA092093F909208131813093FC092093FF
:103B4000FB09228133813093FE092093FD09C7E0F0
:103B5000DAE0D0930602C09305026C97982F88276D
:103B6000840F911D8C010451104048E050E0BE01CB
:103B7000645F7F4F03970E948918A801BE016C5EA5
:103B80007F4F0E948918009709F4ABC6692E782EE2
:103B9000C301809590959093060A8093050A892B1E
:103BA00009F055C68FEF9FEF9B8F8A8F50C680918B
:103BB000BD099091BE0901969093BE098093BD09FD
:103BC0008091ED099927982F88272091EE09820F7F
:103BD000911D8C01045110402DEDA22E29E0B22E32
:103BE00048E050E0B501665E7F4F0E970E9489184D
:103BF000A801B5016E5D7F4F0E9489180097D1F032
:103C0000C92ED82E8FEFC8168FEFD80699F0809165
:103C1000BB099091BC0901969093BC098093BB09A4
:103C20008091C1099091C20901969093C209809335
:103C3000C10950C6C9E0D2E0E091010AF091020A40
:103C40006091FF097091000A4091F7095091F809BD
:103C50002091F9093091FA09898D8823A9F08C8186
:103C60009D81E817F90781F48E819F816817790794
:103C700059F4888199814817590731F48A819B81C9
:103C80002817390709F4B3C1C054DF4F18E0C93C05
:103C9000D10711F308F380910C0A8F73823029F554
:103CA0002091010A3091020A3093400120933F0194
:103CB00010923D0140E0E9E8F9E080819181281708
:103CC000390709F48DC0842F8F5F32968A3011F046
:103CD000482FF3CF80933D018091CB099091CC097F
:103CE00001969093CC098093CB0980910C0A82FDB8
:103CF000F1C58091C5099091C60901969093C609B6
:103D00008093C50984E1F70181A388E290E0909354
:103D1000FB018093FA0180E580A39091060A8091CF
:103D20000A0A838F4091050A8091090A828F468F83
:103D30003091040A8091080A818F358F2091030AFF
:103D400020933D018091070A808F248F9F5F978F7A
:103D5000992361F4842F8F5F868F882339F4832F12
:103D60008F5F858F882311F42F5F248F2091FF09A7
:103D70003091000A3093400120933F018091010A65
:103D80009091020AF701958B848B378B268B80915B
:103D9000F7099091F809F501978F868F8091F909BD
:103DA0009091FA099093FE098093FD098091D909B9
:103DB0009091DA099093F8098093F7098091DB09D3
:103DC0009091DC099093FA098093F90907C59093C3
:103DD0003D0180EC489FE0011124C75FDD4F21C009
:103DE00010923D01E9E0F2E0C0E0D0E090E020E098
:103DF00030E0422F818D882351F3873039F42097AA
:103E000021F0928D8A8D891708F4EF01942F9F5F1E
:103E10002F5F3F4FE054FF4F2A30310551F7909309
:103E20003D01209769F48091C9099091CA090196D2
:103E30009093CA098093C9094DC510923E01BAC03A
:103E4000D0930802C093070283E08A8F888F1E8A6E
:103E500084E08F8B1B8E8091010A9091020A9D83D2
:103E60008C838091FF099091000A9F838E838091BB
:103E7000F7099091F809998388838091F9099091C5
:103E8000FA099B838A8381E0898F809137018C872F
:103E9000809138018D87809139018E8780913A0118
:103EA0008F8781E090E0998B888B8091060A8B87C1
:103EB0008091050A8A878091040A89878091030A84
:103EC0008887809107029091080261E070E008966F
:103ED0000E945018E0910702F09108028091FE01C3
:103EE0008087E0910702F09108028091FF018187AD
:103EF000E0910702F0910802809100028287E09130
:103F00000702F091080280910102838720910B0A39
:103F1000822F9927807F9070813591050CF44CC0D9
:103F200010923D0190913E0140E022952F70332781
:103F300025503040220F331F220F331F34C0DB01C6
:103F4000A352B64FFD0196A9992309F476CF91307B
:103F500011F44F5F28C09230F9F4FD0187A9843035
:103F6000D9F490933E0140933D0120AD3327322F89
:103F7000222781AD9927282B392B3093400120939C
:103F80003F01F2E02B343F0710F02AE432E03B8B94
:103F90002A8B3D8B2C8B10C06352764FFB0187A977
:103FA000882331F0480F642F7727621773073CF29C
:103FB00090933E0140933D0180E180930C0A8091F3
:103FC0000C0A826080930C0A92E09093130A84E0BA
:103FD0008093140A9093150A8AE48093160A8CE25F
:103FE00090E09093FB018093FA0180E6A4C3D09304
:103FF0000802C09307021092020280910C0A482F17
:10400000552742FF03C0198E80E2D9C280910B0A66
:1040100082958F70880F880F80933D012091FA015F
:104020003091FB01281B3109245130403093FB01B2
:104030002093FA01898D8F70823029F4CA018F7321
:1040400090704297F1F0232B21F443705070452B70
:10405000C1F09091030A8885981709F062C3909186
:10406000040A8985981709F05CC39091050A8A852E
:10407000981709F056C39091060A8B85981709F096
:1040800050C380910C0A84FF50C0688979896115FA
:10409000710509F44AC0CE010C960E945018209177
:1040A000070A8091FE01281709F03FC09091080A85
:1040B0008091FF019817C9F59091090A809100023B
:1040C000981799F590910A0A80910102981769F55D
:1040D0002C878091FF018D87809100028E878091CF
:1040E00001028F878B8D8823C9F42E89888D9A8D44
:1040F000891B922F969596959695891B280F2E8B46
:104100003F8987FD8195932F96959695891B830FFF
:104110008F8B269526952695280F288F81E08093F2
:104120000202888D8A8F198A188A898D282F332751
:10413000C9018F7090708430910509F445C28530B3
:10414000910564F48230910509F455C083309105DE
:104150000CF0F8C0019709F0BDC310C0863091057E
:1041600009F4D7C2863091050CF470C287309105EE
:1041700009F4D7C2089709F0ADC31BC280910202AF
:1041800080FFA8C383E0898F80E480930202198AAC
:10419000188A6091FA017091FB016115710509F4AB
:1041A0009AC182E4809302028091070290910802F2
:1041B00008960E945018E0910702F0910802809141
:1041C000FE018087E0910702F09108028091FF01D3
:1041D0008187E0910702F0910802809100028287B6
:1041E000E0910702F091080280910102838773C178
:1041F00010923E015DC08091020280FF98C08091C4
:104200000C0A8F73823109F092C020910B0A822F21
:104210009927807F9070813591050CF44BC01092E6
:104220003D0190913E0140E022952F7033272550AB
:104230003040220F331F220F331F33C0DB01A35244
:10424000B64FFD0196A9992399F2913011F44F5F71
:1042500028C09230F9F4FD0187A98430D9F49093F5
:104260003E0140933D0120AD3327322F222781ADFF
:104270009927282B392B3093400120933F01F2E0FE
:104280002B343F0710F02AE432E03B8B2A8B3D8B26
:104290002C8B10C06352764FFB0187A9882331F025
:1042A000480F642F77276217730744F290933E01FB
:1042B00040933D0183E0898F8091030A8887809134
:1042C000040A89878091050A8A878091060A8B876C
:1042D000809107029091080261E070E008960E94C8
:1042E0005018E0910702F09108028091FE0180874A
:1042F000E0910702F09108028091FF018187E0912F
:104300000702F0910802809100028287E091070283
:10431000F091080280910102838782E48093020277
:10432000198A188A1092FB011092FA01D4C080E217
:10433000809302020E94210FE0910702F09108028F
:10434000118ED3CC80910C0A992780FF4CC024FD9C
:104350004AC088899989892B09F0BCC26091FA0109
:104360007091FB016F5F7F4F80910702909108026F
:1043700008960E945018E0910702F091080280917F
:10438000FE018087E0910702F09108028091FF0111
:104390008187E0910702F0910802809100028287F4
:1043A000E0910702F0910802809101028387209139
:1043B0000202822F8061809302028091FA01909123
:1043C000FB01892B19F02261209302020E94210F28
:1043D00081E090E0998B888B88E0898F1B8E81E14A
:1043E00080930C0AA1C185FF1EC02091110A3327BA
:1043F000322F22278091120A9927282B392B80915E
:10440000050290910602820F931F909306028093FB
:1044100005028091FA019091FB01821B930B90930E
:10442000FB018093FA016091FA017091FB01611523
:10443000710559F1898D84FD28C080910202826046
:1044400080930202809107029091080208960E94D0
:104450005018E0910702F09108028091FE018087D8
:10446000E0910702F09108028091FF018187E091BD
:104470000702F0910802809100028287E091070212
:10448000F091080280910102838780910D0A99279B
:10449000382F222780910E0A280F311D30934001BA
:1044A00020933F018C899D898217930710F0232B5D
:1044B00021F49093400180933F0180913F019091BE
:1044C00040019B8B8A8B80910202992783709070A8
:1044D000892B09F4FFC11092600C10925F0C0E94AE
:1044E000210F80910202282F332725FF07C0109249
:1044F000600C10925F0C198E84E172CF24FF0AC009
:104500001092600C10925F0C81E090E0998B888B88
:1045100084E063CF80915F0C9091600C892B09F14E
:1045200020FF03C0198A188A04C0888999890097D6
:10453000A1F42A893B8980915F0C9091600C281727
:10454000390720F43093600C20935F0C80915F0C4E
:104550009091600C998B888B04C09093600C809331
:104560005F0C1B8E8091FC019091FD0190930602DF
:104570008093050280915F0C9091600C892B59F01B
:1045800088899989009739F088969093FB018093E8
:10459000FA0188E10BC08091020281FF9BC188E291
:1045A00090E09093FB018093FA0180E180930C0AE4
:1045B000C1C08091020280FF8DC1198E80E180937D
:1045C00002020E94210F86C16091FA017091FB01E5
:1045D0006115710519F18091070290910802089602
:1045E0000E945018E0910702F09108028091FE01AC
:1045F0008087E0910702F09108028091FF01818796
:10460000E0910702F0910802809100028287E09118
:104610000702F091080280910102838780910C0AC1
:104620009091020280FF0BC090FF06C087E0898F47
:104630001A8E198A188A3BC086E0898F38C090FF8D
:1046400061C085E0898F198A188A44C16091FA0196
:104650007091FB016115710519F18091070290912C
:10466000080208960E945018E0910702F091080293
:104670008091FE018087E0910702F091080280910D
:10468000FF018187E0910702F0910802809100020A
:104690008287E0910702F0910802809101028387EE
:1046A00080910C0A80FF2EC087E0898F1A8E80913E
:1046B00007029091080261E070E008960E9450188D
:1046C000E0910702F09108028091FE018087E0915D
:1046D0000702F09108028091FF018187E0910702B3
:1046E000F0910802809100028287E0910702F09128
:1046F000080280910102838780E1809302020E9478
:10470000210F0FC08091FA019091FB01892B49F490
:10471000E1C08091020280FFDDC087E0898F1A8EA0
:10472000D9C080E1F70181A388E290E09093FB017A
:104730008093FA0180E580930B0A88858093070AAD
:1047400089858093080A8A858093090A8B858093DE
:104750000A0A8C858093030A8D858093040A8E85CE
:104760008093050A8F858093060A86E08093F4097A
:104770008C819D819093000A8093FF098E819F8197
:104780009093020A8093010A8091D9099091DA09E5
:104790009093F8098093F7098091DB099091DC09E7
:1047A0009093FA098093F909888199819093FC0983
:1047B0008093FB098A819B819093FE098093FD0978
:1047C000898D84FF05C010920E0A10920D0A06C052
:1047D00082E080930D0A8AE480930E0ACBEED9E042
:1047E00080E48093F3098091FA019091FB01892F75
:1047F00099278093ED092091FA012093EE091092F8
:10480000120A1092110A1092100A10920F0A982F91
:104810008827820F911D8C010451104048E050E020
:10482000BE01645F7F4F0E970E948918A801BE01E8
:104830006C5E7F4F0E948918009719F40FEF1FEFED
:1048400002C0092F182F009510951DA30CA3CBEEC5
:10485000D9E085E48093EB091092EC091092F209FB
:104860001092F10980913501909136010196909353
:10487000360180933501292F33272093EF09809348
:10488000F0091092F6091092F50944E150E0BE01DA
:1048900080E090E00E948918009719F40FEF1FEF55
:1048A00002C0092F182F009510951B870A87809149
:1048B000BF099091C00901969093C0098093BF09E8
:1048C0008091A5099091A60901969093A6098093DD
:1048D000A50904C01092FB011092FA011092020285
:1048E00005C01092060A1092050A5CC9DF91CF91AB
:1048F0001F910F91FF90EF90DF90CF90BF90AF90FE
:104900009F908F907F906F900895CF93DF93CDED20
:10491000D9E06091FB097091FC092FEF6F3F72079E
:1049200089F48091FD099091FE098F5F9F4F51F4AA
:10493000DE01EEE1F1E086E001900D92815009F494
:10494000D6C0FACF8091D5099091D609AB01482302
:1049500059232091D9093091DA09822393234817EA
:104960005907A1F4E091FD09F091FE098091D70962
:104970009091D809AF01482359232091DB09309148
:10498000DC09822393234817590789F080919D09F8
:1049900090919E0990939A018093990180919F092B
:1049A0009091A00990939C0180939B0108C0709303
:1049B0009A0160939901F0939C01E0939B011092FE
:1049C0009D016091990170919A0140919B015091D4
:1049D0009C0130E020E081E491E0FC018081918144
:1049E0006817790731F4828193814817590709F4D0
:1049F00074C0232F2F5FCF010B96283011F0322F78
:104A0000ECCF20939D01283009F069C046E050E0CA
:104A10006FEF70E08DED99E00E94242CEDEFF9E04E
:104A200086E0DF011D928A95E9F77A97AFE2B1E05F
:104A300086E00D9001928150E1F7A3EFB9E0EFE23B
:104A4000F1E086E001900D928150E1F780919901AB
:104A500090919A019FA38EA380919B0190919C01BC
:104A60009093060A8093050A8091D9099091DA09FA
:104A70009D8F8C8F8091DB099091DC099093FC09CC
:104A80008093FB0980E091E09093F2098093F10913
:104A90009093EC098093EB0988E090E09093EE0905
:104AA0008093ED0986E08093EF0984E08093F0091C
:104AB00088E096E09093EA098093E90983E19AE01F
:104AC00090930602809305028AE290E09093FB01A6
:104AD0008093FA0181E090E024C020939D01ADED28
:104AE000B9E0349686E001900D928150E1F7A3EE93
:104AF000B9E0EFE2F1E086E001900D928150E1F73C
:104B000088E090E09093EA098093E9098091FA01A6
:104B10009091FB010E969093FB018093FA0180E047
:104B200090E0DF91CF91089580919F018F5F8093F6
:104B30009F0110929D0190E07BE0482F552760E097
:104B4000979FF0011124EF5BFE4F808191812281BC
:104B50003381822B932B892B59F082859A01281B54
:104B600031092837310524F0108211821282138214
:104B7000962F9F5F692F983018F390939D010895A9
:104B800010929D0190E02BE080E0929FF0011124B3
:104B9000EF5BFE4F10821182128213828F5F982F7B
:104BA000883098F388E080939D010895FF920F93D9
:104BB0001F93CF93DF938091FA019091FB018A9725
:104BC00028F41092FB011092FA01C2C11092FB016D
:104BD0001092FA010DED19E08091F1099091F2091E
:104BE00021E08030920741F08050924009F0B0C13E
:104BF00000C130939D0196C02091030A3091040AB0
:104C00008091D9099091DA092817390709F0A0C1D4
:104C10002091050A3091060A8091DB099091DC0908
:104C20002817390709F094C110929D0160E070E0E7
:104C3000A1E4B1E0E091F909F091FA094091FB0992
:104C40005091FC09F0909F012D913C9111972115F5
:104C50003105C9F0ED018A819B810097A1F0E2172F
:104C6000F30789F44817590771F470939D01FD010A
:104C70003496C3EFD9E086E0099001928150E1F7C4
:104C8000FD01F28666C06F5F1B96683011F0762FCB
:104C9000DBCF10929D0120E030E081E491E0EC0157
:104CA00088819981892B29F48A819B81892B09F438
:104CB000A0CF2F5FCE010B96283011F0322FEFCF0F
:104CC00020939D01283071F51092A00110929E0151
:104CD00010929D01B0919F01CB2FDD2770E0A0E0E5
:104CE00040E050E0EBE4F1E060819E01261B3109D9
:104CF0008A2F9927821793071CF4AB2FA61B742FBA
:104D00004F5F5F4F3B964830510571F770939E019E
:104D1000A093A00170939D018BE0789FE001112486
:104D2000CF5BDE4F8091F9099091FA09A091FB09C0
:104D3000B091FC09FE0181939193A193B193A3EFEC
:104D4000B9E086E00D9001928150E1F780919F01DA
:104D50008A8780E092E0E8019D8B8C8BEDEFF9E093
:104D6000DF011A9786E00D9001928150E1F7A3EFE1
:104D7000B9E0EFE2F1E086E001900D928150E1F7B9
:104D8000A3EEB9E0EFE2F1E086E001900D928150F0
:104D9000E1F7EDEDF9E0DF01909686E00D900192EC
:104DA0008150E1F78091F9099091FA09F80197A3F0
:104DB00086A38091FB099091FC0991A780A780911F
:104DC000D9099091DA09958F848F8091DB099091B0
:104DD000DC09978F868F88E096E0958784878AE242
:104DE00090E09093FB018093FA01B2C030939D0153
:104DF00098C02091030A3091040A8091D9099091BA
:104E0000DA092817390709F0A3C02091050A309163
:104E1000060A8091DB099091DC092817390709F00F
:104E200097C010929D01F0E0E1E0A1E4B1E0609153
:104E3000F9097091FA094091FB095091FC09109110
:104E40009F012D913C91119721153105C9F0ED017C
:104E50008A819B810097A1F06217730789F4481734
:104E6000590771F4F0939D01FD013496C3EFD9E029
:104E700086E0099001928150E1F7FD01128768C038
:104E80008E2F8F5F1B96893019F0FE2FE82FD9CF18
:104E900010929D0120E030E081E491E0EC018881F6
:104EA0009981892B29F48A819B81892B09F49ECFD2
:104EB0002F5FCE010B96283011F0322FEFCF2093C9
:104EC0009D01283071F51092A00110929E01109260
:104ED0009D01B0919F01CB2FDD2770E0A0E040E065
:104EE00050E0EBE4F1E060819E01261B31098A2F3E
:104EF0009927821793071CF4AB2FA61B742F4F5FC3
:104F00005F4F3B964830510571F770939E01A09317
:104F1000A00170939D018BE0789FE0011124CF5B8D
:104F2000DE4F8091F9099091FA09A091FB09B091A7
:104F3000FC09FE0181939193A193B193A3EFB9E092
:104F400086E00D9001928150E1F780919F018A8760
:104F5000DF91CF911F910F91FF900895FC018289FD
:104F6000938920893189821B930B0895FC018485E4
:104F70009585892B19F081E090E00895848982302D
:104F800029F483E0848B80E090E008958091020210
:104F90009927969587958170907008951F93CF9368
:104FA000DF93EC018A819B81009729F0803D910578
:104FB00009F05CC012C04115510529F41B821A8208
:104FC00082E090E05FC07D836C835B874A871C8AA8
:104FD00047C080ED90E09B838A838C89863019F0EE
:104FE00080E090E027C080910202992780FF46C0B0
:104FF0008A859B85E0910702F091080242895389D6
:105000002C813D814817590758F4841B950B9B87C9
:105010008A8782899389280F391F3D832C8306C094
:10502000280F391F3D832C831B861A8681E08C8BC9
:1050300081E090E0182F8A859B85E0910702F0912E
:105040000802628973892C813D816817790708F00D
:10505000BC01C9010E941B1986E08C8B10FF0BC09C
:105060008A859B85892B09F0B4CF1C8A1B821A8202
:1050700083E090E007C080E090E004C082FFFBCFB7
:1050800010E0D9CFDF91CF911F910895FC01148AD0
:105090001586148671876087538B428B7787668766
:1050A000518B408B118210821382128208950F93CC
:1050B0001F93CF93DF93EC018A819B81009729F0A6
:1050C0008753914009F094C010C02A893B89888594
:1050D00099859F878E87398B288B8C859D85892B19
:1050E00001F587E391E09B838A838C859D85892BDD
:1050F00051F48C89823019F483E08C8B76C08091D6
:10510000020281FF72C082E08C8B80910502909137
:1051100006029F838E838091FA019091FB019D8707
:105120008C878E01025F1F4F2C853D85F8014281DF
:10513000538124173507F8F46E817F81A9018E858C
:105140009F850E94052C8E859F852C853D85820F2D
:10515000931F9F878E87F80182819381821B930B17
:10516000938382838E819F81820F931F9F838E837F
:105170001D861C86B2CF8E859F856E817F81241708
:105180003507B1F40E94052C8E859F852C853D85C1
:10519000820F931F9F878E87F801138212828E8160
:1051A0009F81820F931F9F838E831D861C8625C03F
:1051B0000E94052C8E859F85F80122813381820F04
:1051C000931F9F878E878C859D85821B930B9D8760
:1051D0008C878E819F81820F931F9F838E83138282
:1051E00012820BC01C8A1B821A8280E090E00DC0E4
:1051F0001B821A8283E090E008C02A893B89888953
:1052000099892817390771F3F3CFDF91CF911F9157
:105210000F9108951F93CF93DF93DC01162FEC01BC
:105220008A819B81009729F08C51914009F07EC0C2
:1052300012C0ED012A893B89888599859F878E87D1
:10524000398B288BFD0184859585892B11F58CE19F
:1052500091E093838283ED018C859D85892B51F4A8
:105260008C89823019F483E08C8B5DC080910202BE
:1052700081FF59C082E0FD01848B809105029091ED
:105280000602978386838091FA019091FB019587AE
:105290008487ED012E96AD014A5F5F4FBD01645FCB
:1052A0007F4F20C0FA0180819181FC012081E8813B
:1052B000F9812083FA018081918101969183808315
:1052C00088819981019699838883FB0180819181EE
:1052D0000197918380838A819B8101979B838A8335
:1052E000211751F18A819B81FB0120813181892B1A
:1052F00089F0232BB9F6A6CFEA01E881F9818191E3
:1053000021503040EB0139832883EA01F983E88397
:10531000811791F02115310509F494CFEDCFFD01EE
:10532000148A1382128280E090E00FC0ED011B828C
:105330001A8283E090E009C0FD01228933898089C7
:1053400091892817390759F3F1CFDF91CF911F9138
:105350000895CF92DF92FF920F931F93CF93DF9325
:10536000EC018B016A018A819B81009729F08F3EB5
:10537000910509F069C01FC06115710529F41B82F0
:105380001A8282E090E06CC0CA01FB0109959B87FC
:105390008A8780910502909106029D838C831C8AE6
:1053A0008091020282FF03C0C601F80109958FEEC9
:1053B00090E09B838A838C89863019F080E090E0AE
:1053C00027C080910202992780FF46C08A859B856D
:1053D000E0910702F0910802428953892C813D81B6
:1053E0004817590758F4841B950B9B878A87828935
:1053F0009389280F391F3D832C8306C0280F391F3E
:105400003D832C831B861A8681E08C8B81E090E0A3
:10541000F82E8A859B85E0910702F0910802628947
:1054200073892C813D816817790708F0BC01C90197
:105430000E941B1986E08C8BF0FE0BC08A859B8531
:10544000892B09F0ADCF1C8A1B821A8283E090E081
:1054500007C080E090E004C082FFFBCFFF24D9CFDB
:10546000DF91CF911F910F91FF90DF90CF90089522
:10547000A8E1B0E0EEE3FAE20C94DD32222E332E06
:10548000442E552E662E772E882E992E002309F451
:105490006EC0FE01719688E0DF011D928A95E9F7E2
:1054A000DE01119688E001900D928150E1F729828A
:1054B0003A824B825C826D827E828F829886E0E2A5
:1054C000E01B1E16CCF529813A814B815C81602F4F
:1054D000772767FD7095DA01C901062E04C0880F91
:1054E000991FAA1FBB1F0A94D2F789879A87AB8797
:1054F000BC8704C05695479537952795EA95D2F70E
:105500008D819E81AF81B88504C0880F991FAA1F25
:10551000BB1F6A95D2F7282B392B4A2B5B2B2D8783
:105520003E874F87588B29843A844B845C846D84F2
:105530007E848F8498881BC019861A861B861C86D9
:105540002E2F332727FD3095309521953F4F8981A8
:105550009A81AB81BC8104C0880F991FAA1FBB1F11
:105560002A95D2F78D879E87AF87B88BDCCF222D07
:10557000332D442D552D662D772D882D992DE2E163
:1055800068960C94F932CF93DF93AC01029710F434
:1055900042E050E0A091BD0CB091BE0CFD01C0E016
:1055A000D0E020E030E020C0808191818417950711
:1055B00069F482819381209719F09B838A8304C0C8
:1055C0009093BE0C8093BD0CCF0132C04817590791
:1055D00038F42115310519F08217930708F49C015E
:1055E000EF010280F381E02D3097F1F621153105AE
:1055F00089F1C901841B950B049708F4A901E0E027
:10560000F0E026C08D919C91119782179307E9F4E1
:105610004817590779F4ED018A819B81309719F079
:105620009383828304C09093BE0C8093BD0CCD0104
:10563000029649C0841B950BFD01E80FF91F4193A9
:10564000519302978D939C933AC0FD01A281B3813F
:105650001097C1F68091BB0C9091BC0C892B41F442
:1056600080912601909127019093BC0C8093BB0CF4
:1056700020912801309129012115310541F42DB7E0
:105680003EB78091240190912501281B390BE091B0
:10569000BB0CF091BC0C2E1B3F0B2417350788F078
:1056A000CA0102962817390760F0CF01840F951FB1
:1056B00002969093BC0C8093BB0C41935193CF0105
:1056C00002C080E090E0DF91CF910895CF93DF9307
:1056D000009709F44EC0EC0122971B821A82A09118
:1056E000BD0CB091BE0C109711F140E050E001C02C
:1056F000DC01AC17BD0700F1BB83AA83FE01219139
:105700003191E20FF31FEA17FB0771F42E5F3F4F51
:105710008D919C911197820F931F99838883FD012E
:10572000828193819B838A834115510559F4D093DB
:10573000BE0CC093BD0C1DC0FD0182819381AD01E3
:105740000097B1F6FA01D383C28321913191E20F20
:10575000F31FEC17FD0769F42E5F3F4F8881998195
:10576000820F931FFA01918380838A819B819383A7
:105770008283DF91CF910895FB01DC0140FF05C0DA
:1057800002C005900D9205900D9242505040C8F70E
:105790000895FC0105900020E9F7809590958E0F03
:1057A0009F1F0895FB01DC014150504078F08D911E
:1057B0000590202D302D3062313624F03B3714F423
:1057C00020628062821B19F4002071F7881B990BFC
:1057D0000895FB01DC014150504048F005900D92C6
:1057E0000020C9F701C01D9241505040E0F70895D4
:1057F000FC014150504030F001900616D1F731972E
:10580000CF010895882799270895FB01DC0140FF07
:1058100005C002C001900D9201900D92425050407F
:10582000C8F708956817790768F4FB01DC01E40FF5
:10583000F51FA40FB51F02C002900E9241505040B8
:10584000D8F708950C94052CDC0140FF03C001C07B
:105850006D936D9342505040D8F70895FC0101902C
:10586000061629F00020D9F788279927089531973F
:10587000CF0108950F931F93CF93DF93CDB7DEB77A
:1058800060970FB6F894DEBF0FBECDBF0F89188D9D
:10589000898D9A8D97FF03C08FEF9FE701C0019715
:1058A00098878F831C830B838EE08E83AE01435ECB
:1058B0005F4F5A8349836B8D7C8DCE0103960E9486
:1058C000CC2C2F813885821793070CF49C01020F92
:1058D000131FF801108260960FB6F894DEBF0FBE5A
:1058E000CDBFDF91CF911F910F9108950F931F931B
:1058F000CF93DF93CDB7DEB760970FB6F894DEBFD6
:105900000FBECDBF0F89188D8EE08E831C830B8355
:105910008FEF9FE798878F83AE01455E5F4F5A8375
:105920004983698D7A8DCE0103960E94CC2C2985FE
:105930003A85020F131FF801108260960FB6F89493
:10594000DEBF0FBECDBFDF91CF911F910F910895A4
:10595000CF93DF93CDB7DEB760970FB6F894DEBF75
:105960000FBECDBF8DE08E838D899E899C838B83F6
:10597000AE01475E5F4F5A8349836F89788DCE01B0
:1059800003960E94812F60960FB6F894DEBF0FBE7B
:10599000CDBFDF91CF9108952F923F924F925F92AA
:1059A0006F927F928F929F92AF92BF92CF92DF922F
:1059B000EF92FF920F931F93CF93DF93CDB7DEB794
:1059C00062970FB6F894DEBF0FBECDBF882499242E
:1059D00054012C017A8B698B3A01FC0117821682E3
:1059E000838181FD03C08FEF9FEF72C2CC24DD2441
:1059F0005EC2C0FE45C2832D80538A30E0F4F0E3DE
:105A00003F1641F42D85222329F4C3FC03C080E016
:105A100091E078C08AE0ED85E802C0011124380EDB
:105A2000F32DF053FD87F7FF02C02FE72D87C3FC4E
:105A300039C22D8437C2C60188709070C3FE05C07C
:105A40003D85332311F4E1E0ED87F7E6F3156CF1C2
:105A500025E632160CF067C033E5331609F487C02B
:105A60003315BCF08BE2381609F441C083154CF0B5
:105A700090E2391609F43FC0E3E23E1609F0F6C1A0
:105A800044C0FDE23F16E1F12EE2321609F0EEC10C
:105A900041C033E6331609F44CC033150CF480C012
:105AA00088E5381609F0E2C11FC0E0E73E1609F4A8
:105AB000A1C0E3155CF0FCE63F1691F12FE632162B
:105AC00089F039E6331609F0D1C16AC0E5E73E1620
:105AD00009F498C0F8E73F1639F023E7321609F0C9
:105AE000C5C12FC038E08DC080E1888B8BC0E0E15C
:105AF000F0E0CE2ADF2A20E230E0C22AD32AD2C147
:105B000080E890E0C82AD92ACDC1E0E4F0E0CE2AAE
:105B1000DF2AC8C128E030E0C22AD32A1D86C2C1CC
:105B200084E090E0EFCF5FE3852E2A9443E6342EA5
:105B300033C1F30180802A9422E030E0620E731EAC
:105B40002BC1F30180809180892B49F0FD856F2F57
:105B5000772767FD7095C4010E94323219C0F401A5
:105B600001900020E9F73197E819E88B12C0F301A2
:105B700080809180892B49F0FD856F2F772767FD05
:105B80007095C4010E94273203C0C4010E94C92B32
:105B9000888B22E030E0620E731E3889231AFCC025
:105BA000C2FE08C0F30180819181A281B38124E00B
:105BB00030E009C0F30180819181AA2797FDA0956B
:105BC000BA2F22E030E0620E731E4C015D01B7FF78
:105BD0000CC082E090E0C82AD92AB094A094909496
:105BE0008094811C911CA11CB11CEFEBFFEFCE2215
:105BF000DF2221C020E430E0C22AD32A38E7332E46
:105C000030E1388BC2FE08C0F30180819181A2810E
:105C1000B38124E030E007C0F30180819181AA279D
:105C2000BB2722E030E0620E731E4C015D018FEC59
:105C30009FEFC822D92285017401FE013196FF87AA
:105C4000EE87F8898F2E9924AA24BB24C801B701B6
:105C5000A50194010E9473336A301CF0630D6152F8
:105C600001C0605DEE85FF856193FF87EE87C80107
:105C7000B701A50194010E94733379018A012115AE
:105C800031054105510511F7882499245401CE01AD
:105C900001968E84881AC60182739070892B09F050
:105CA0002A94C6FE07C0F889F03111F482E001C0E1
:105CB00081E0281A28E0E22EF12CEC20FD20C3FE22
:105CC00016C08D85282F332727FD3095882D9927DD
:105CD000821793073CF0E7EFFFEFCE22DF22EE249E
:105CE000FF2405C0FD85F819FD872F1A01C028186B
:105CF000C60180789170892B69F4822D06C0B201AB
:105D000080E290E00E948032812F182F11501816E7
:105D1000B4F3212EC1FE04C0B2018DE290E00BC0AD
:105D2000C4FE04C0B2018BE290E005C0C5FE05C010
:105D3000B20180E290E00E948032C6FE0FC0B20144
:105D400080E390E00E9480322889203139F4B2014A
:105D5000832D992787FD90950E948032D0FE0DC03B
:105D6000822D06C0B20180E390E00E948032812F34
:105D7000182F11501816B4F3212EEF2869F02D8535
:105D800006C0B20180E390E00E948032212F122FE2
:105D900011501216B4F31D8790E8E92EF12CEC2077
:105DA000FD20C7FC0DC0822D06C0B20180E290E04C
:105DB0000E948032812F182F11501816B4F3212E13
:105DC00033E6331641F4B201882D992787FD90956B
:105DD0000E9480323BC083E7381689F4840109C0F1
:105DE000F80181918F01B201992787FD90950E945A
:105DF0008032F889F150F88BFF3F91F715C023E509
:105E0000321619F00E851F851AC0840108C0F801EA
:105E10008491B20199270E9480320F5F1F4FF88949
:105E2000F150F88BFF3F99F7480110C0F8018291BB
:105E30008F01B201992787FD90950E948032CE0193
:105E400001960817190791F71F870E87EF28A9F009
:105E5000822D06C0B20180E290E00E948032812F44
:105E6000182F11501816B4F3212E07C0B201832D3C
:105E7000992787FD90950E948032CC24DD2412C0A2
:105E8000F5E23F1641F42AE0288B22241D8681E0AA
:105E9000C82ED12C07C0B201832D992787FD90957C
:105EA0000E94803289899A8901969A8B898BF201A6
:105EB000838183FF04C0E989FA89349003C0E989AA
:105EC000FA893080332009F094CDF20186819781E0
:105ED00062960FB6F894DEBF0FBECDBFDF91CF91B3
:105EE0001F910F91FF90EF90DF90CF90BF90AF90F8
:105EF0009F908F907F906F905F904F903F902F90EA
:105F000008952F923F924F925F926F927F928F925D
:105F10009F92AF92BF92CF92DF92EF92FF920F9338
:105F20001F93CF93DF93CDB7DEB72A970FB6F894C0
:105F3000DEBF0FBECDBFAA24BB2465013C017A871A
:105F400069872A01FC0117821682838180FD05C0C2
:105F50002FEF3FEF3D832C835FC21F821E824FEFE6
:105F60005FEF5D834C83882499241B821A821982F7
:105F70001DC25981E52EFF24E0FEDBC1153219F464
:105F80005E7F598300C2912F90539A3060F48FE75F
:105F9000281611F480E004C08AE0289E802D112488
:105FA000282E290EFEC1812F992787FD90950E94EA
:105FB0002D33382E9EE6391609F48CC19315DCF08A
:105FC000A8E63A1609F4EDC1A31564F0B3E63B1652
:105FD00091F1E4E63E1609F4A2C0FAE23F1609F098
:105FE00088C121C029E6321609F499C03CE633166F
:105FF00009F07FC11CC043E7341609F44BC04315B8
:106000004CF05FE6351609F47FC080E7381609F0DA
:1060100070C180C095E7391609F47EC0A8E73A162A
:1060200009F067C177C0B981B061B983BAC1E981AC
:10603000E460E983B6C1870100711070E4FC07C019
:10604000D201AD90BC90E2E0F0E04E0E5F1EFFE7A3
:106050002F1611F431E0232E75010FC0C3010E94E9
:106060003D324C012FEF8F3F920709F4D1C101154A
:10607000110519F4D7018D937D012A94822D8F5F2C
:10608000181664F3570135C15701B301C4010E94CA
:10609000AD3234C0870100711070E4FC07C0F2011A
:1060A000A080B18022E030E0420E531EC3010E9466
:1060B0003D324C010E941E33892BC1F73FEF8316FE
:1060C0003FEF930609F4A4C1750112C0C4010E94F8
:1060D0001E33892BC9F60115110519F4D7018D92CC
:1060E0007D01C3010E943D324C018F5F9F4F29F01B
:1060F0002A94822D8F5F18164CF35701012B09F05B
:10610000F8C0F5011082F5C0E981E260E983F8E0AA
:10611000F88705C020E12887398132603983C301BF
:106120000E943D324C010E941E33892BC1F74FEF74
:1061300084164FEF940609F447C1882D8D3211F073
:106140008B3299F42A9412140CF03EC18D3219F45A
:10615000598158605983C3010E943D324C018FEF31
:1061600088168FEF980609F42FC190E38916A1F5E0
:10617000AA24BB2465012A9412140CF07EC0C3012A
:106180000E943D324C01AFEF8F3F9A0709F475C072
:106190000E942D338837D9F4BFE63B1631F0E4E690
:1061A0003E1619F0F5E73F1629F4B301C4010E9429
:1061B000AD3263C0C3010E943D324C018F5F9F4FDF
:1061C00019F430E1388759C040E1488705C059E6E5
:1061D000351611F488E08887EE24FF248701C40176
:1061E0000E942D3320EDC22E2FEFD22EC80ED91EC5
:1061F0009AE0C916D1043CF0C601C19762F0A9ED3E
:10620000BFEFCA0EDB1ED7FC06C0B8858B2F9927BF
:10621000C816D9063CF057016801B301C4010E94B9
:10622000AD3221C0E8852E2F332744275527C801DA
:10623000B7010E9454337B018C01C601AA2797FD48
:10624000A095BA2FE80EF91E0A1F1B1F2A941214DC
:1062500044F4C3010E943D324C018F5F9F4F09F00F
:10626000BECF57016801298123FF07C0AA24BB24A0
:106270006501AE18BF08C00AD10A4981242F33270F
:1062800024FD37C0C90186709070069741F4D20191
:10629000ED91FC91A082B182C282D38226C021FFFF
:1062A00006C0D201ED91FC91B182A0821EC0C20154
:1062B000029622FF08C0D201ED91FC91A082B1822A
:1062C000C282D38205C0D201ED91FC91B182A0823D
:1062D0002C010FC0E4FC0DC0F20120813181F301DB
:1062E00086819781D9018D939C93E2E0F0E04E0E78
:1062F0005F1EF301868197812A813B812817390728
:106300006CF4398134FD06C04E815F814F5F5F4F71
:106310005F834E831D821C82198243C05EE6351660
:1063200009F052C08FEF88168FEF980609F44CC021
:10633000F3CF153269F4F3010680F781E02DFB837A
:10634000EA83FAE0F8878FE7282E21E0298329C025
:10635000812F992787FD90950E941E33892B99F0F4
:10636000C3010E943D324C010E941E33892BC1F7AC
:106370003FEF83163FEF930609F441C0B301C40118
:106380000E94AD320EC0C3010E943D324C018F5FAE
:106390009F4FD1F0812F992787FD909588169906F8
:1063A00099F489859A8501969A878987F301838173
:1063B00083FF04C0E985FA85149103C0A985BA85D5
:1063C0001C91112309F0D5CDB9812B2F332720FF44
:1063D00011C0F301868197814A815B814817590773
:1063E0004CF424FD05C08E819F8101969F838E838E
:1063F0001D821C829FEF89169FEF990621F4AE81C2
:10640000BF81AB2B49F0EE81FF81FD83EC8304C09B
:10641000F9812F2F3327DDCF8C819D812A960FB6EE
:10642000F894DEBF0FBECDBFDF91CF911F910F91CA
:10643000FF90EF90DF90CF90BF90AF909F908F90A4
:106440007F906F905F904F903F902F900895FC0148
:106450000590615070400110D8F7809590958E0F8F
:106460009F1F0895FC016150704001900110D8F702
:10647000809590958E0F9F1F0895CF93DF93EC0129
:106480002B81822F992780FF15C086FF0AC02F7BA2
:106490002B838E819F8101969F838E838A8199278A
:1064A0002CC082FF12C0E881F9818081882329F401
:1064B00020622B838FEF9FEF20C0282F332727FDEB
:1064C00030953196F983E88311C0EA85FB85CE01CA
:1064D00009959C0197FF0AC08B812F5F3F4F11F4F4
:1064E00090E101C090E2892B8B83E4CF8E819F8164
:1064F00001969F838E83822F9927DF91CF910895F4
:106500000F931F93CF93DF938C01EB018B8199271E
:1065100081FF1BC082FF0DC02E813F818C819D8138
:106520002817390764F4E881F9810193F983E88336
:1065300006C0E885F985802F0995892B31F48E8175
:106540009F8101969F838E8302C00FEF1FEFC801CA
:10655000DF91CF911F910F910895AC01FB01238131
:10656000822F992780FF12C086FD10C08FEF4F3F0A
:10657000580761F0428320642F7D238386819781B1
:10658000019797838683842F992708958FEF9FEF34
:106590000895AA1BBB1B51E107C0AA1FBB1FA6176A
:1065A000B70710F0A61BB70B881F991F5A95A9F7BC
:1065B00080959095BC01CD0108952F923F924F9206
:1065C0005F926F927F928F929F92AF92BF92CF9283
:1065D000DF92EF92FF920F931F93CF93DF93CDB78C
:1065E000DEB7CA1BDB0B0FB6F894DEBF0FBECDBF04
:1065F00009942A88398848885F846E847D848C84D5
:106600009B84AA84B984C884DF80EE80FD800C81DD
:106610001B81AA81B981CE0FD11D0FB6F894DEBFC0
:106620000FBECDBFED0108951ED001921A94E1F77F
:106630000895019020D01A94E1F70895911127C090
:10664000803251F08A3041F08C3031F08D3021F0C1
:10665000893011F08B3099F708958F931DD08F9169
:1066600009F080620895F999FECFB2BDA1BDF89AF4
:10667000119600B40895F999FECFB2BDA1BD00BC3A
:1066800011960FB6F894FA9AF99A0FBE08959927C1
:106690008827089585FDFBCF80629111F8CF813660
:1066A000ECF38B37DCF70895629FD001739FF00104
:1066B000829FE00DF11D649FE00DF11D929FF00D92
:1066C000839FF00D749FF00D659FF00D9927729FC9
:1066D000B00DE11DF91F639FB00DE11DF91FBD0154
:1066E000CF0111240895A1E21A2EAA1BBB1BFD01A4
:1066F0000DC0AA1FBB1FEE1FFF1FA217B307E407A1
:10670000F50720F0A21BB30BE40BF50B661F771FF8
:10671000881F991F1A9469F76095709580959095D8
:0A6720009B01AC01BD01CF010895FB
:10672A0000F8200023002600290021002400270069
:10673A002A0000FF030F2200250028002B00FFFF7C
:0A674A00FFFFFFFF2000BF0C00005E
:00000001FF
